:100000001DEF12F069EF12F0046ED8CF05F0E0CFCB
:1000100006F00001E9CF0CF0EACF07F0E1CF08F0DD
:10002000E2CF09F0D9CF0AF0DACF0BF0F3CF12F01C
:10003000F4CF13F0FACF14F0F5CF15F0F6CF16F099
:10004000F7CF17F000C00EF001C00FF002C010F0A3
:1000500003C011F0F2AA30EF00F0F2B47EEF00F02E
:100060000EC000F00FC001F010C002F011C003F08C
:100070000CC0E9FF07C0EAFF078E08C0E1FF09C016
:10008000E2FF0AC0D9FF0BC0DAFF12C0F3FF13C0B2
:10009000F4FF14C0FAFF15C0F5FF16C0F6FF17C035
:1000A000F7FF045006C0E0FF05C0D8FF10000A01AA
:1000B000675302E1899201D08982000112000A018E
:1000C0006751F80B12E1928E67A102D08B8401D0A8
:1000D0008B9467A302D08B8201D08B9267A502D04C
:1000E000898C01D0899C898607D08996685302E063
:1000F000898E01D0899E929E00011200D76A070E58
:10010000D66E0A01616B80BE612B6153D8B441D1B8
:100110000901B053D8B402D00A013BD1B3511B5CE2
:10012000D8B4C8D01BC0B3F9898A1B50010A00019A
:1001300014E0030A12E0010A2CE0070A3DE0010A7C
:100140004FE0030A61E0010AD8B472D00F0AD8B4B4
:1001500083D0010AD8B494D0A7D0010E0A01676FEA
:100160000001A5DF0A016769686B0001A8DF070EBF
:100170000A01676F686B0001A2DF1B2C05D0090123
:10018000A66B020EA56F04D00901A66B140EA56F15
:100190008CD00A01676B00018ADF0A016769686B0E
:1001A00000018DDF0A01676B686B000188DF0901C0
:1001B000A66B020EA56F79D00A01676B000177DF8D
:1001C0000A016769686B00017ADF020E0A01676F36
:1001D000686B000174DF0901A66B020EA56F65D084
:1001E0000A01676B000163DF0A016769686B000140
:1001F00066DF030E0A01676F686B000160DF0901AB
:10020000A66B020EA56F51D00A01676B00014FDF8C
:100210000A016769686B000152DF060E0A01676F09
:10022000686B00014CDF0901A66B020EA56F3DD083
:100230000A01676B00013BDF0A016769686B000117
:100240003EDF050E0A01676F686B000138DF0901A8
:10025000A66B020EA56F29D00A01676B000127DF8C
:100260000A016769686B00012ADF040E0A01676FE3
:10027000686B000124DF0901A66B020EA56F15D083
:100280000A01676B000113DF0A016769686B0001EF
:1002900016DF070E0A01676F686B000110DF0901A6
:1002A000A66B020EA56F01D00901899AA86BA76BF6
:1002B000A46BA36B80AA25D0899AAF5315E0CE50CA
:1002C0009F6FCFCFA0F9A2C99AF9A1C999F9A0C986
:1002D00098F99FC997F9A0C99EF99FC99DF9A2C92C
:1002E0009CF9A1C99BF9AF6BCF6ACE6AA26BA16BD7
:1002F000A06B9F6BB26BB16BA46BA36BA86BA76B6E
:1003000003D0A32BD8B4A42B1B50010A000111E089
:10031000030A0FE0010A18E0070A16E0010A14E0D8
:10032000030A12E0010A10E00F0A0EE0010A0CE0D5
:100330002ED00901A551A35D06E1A651A45D03E1FC
:10034000898A010EAF6F24D00901A551A35D1EE17A
:10035000A651A45D1BE1A851020809E2FF0A03E1CE
:10036000A751E80804E2898A010EAF6F0FD0A551AA
:10037000200809E1A65307E11B50090801E01B2AE8
:10038000A86BA76B03D0D890A537A63701D0090179
:100390000A0180A805D00901A92BD8B4AA2B03D043
:1003A0000901AA6BA96BA8510A080BE2FF0A03E135
:1003B000A751B80806E21B50030801E01B06A86B12
:1003C000A76BA72BD8B4A82B61CAB0F9CE500A01ED
:1003D000656FCFCF66FA66510901B25D0CE308E1A3
:1003E000B1510A01655DD8A002D0090104D009010C
:1003F000A12BD8B4A22B66CAB2F965CAB1F90A0119
:10040000616B81B8612B615306E10901AD5302E0D4
:10041000010EAB6F0A0161CAADF9616B81BA612B44
:10042000615306E10901AE5302E0010EAC6F0A010F
:1004300061CAAEF9F294000130EF00F0445254204A
:100440005265733130487A2020004452542052655E
:10045000732031487A20200052435020446976208E
:100460003120202020005243502044697620313032
:100470002020200052435020446976203130302023
:1004800020005243502044697620316B2020200008
:10049000524350204469762031306B202000524373
:1004A0005020446976203130306B20005243502078
:1004B00044697620314D20202000204558543A00D0
:1004C00020494E543A0046524551203A2573487A05
:1004D000202000006D616B65207461626C65000016
:1004E000434F554E543A25386C6400004359434CF1
:1004F000453A25326C642054286D73293A25346CB2
:100500006400090EEA6EEC0EE96EEF500EE0140E78
:10051000016E006A002EFED7012EFBD7BF0E006EC3
:10052000002EFED700D0EF2EF2D71200FF0E926EF3
:10053000936E946E949694989394949A93969390C1
:10054000929A898A870ECD6ECC6A92908990929207
:10055000898294949492929C92968986899492949A
:100560006168F19E57EF12F00A0123A902D08B8631
:1005700001D08B9623A702D08A8001D08A9023A530
:1005800002D08A8601D08A9623A302D08B8A01D01A
:100590008B9A23A102D08A8401D08A940001120090
:1005A0008B8800D08B9800D01200640E0901EC6F8C
:1005B0000001A7DF030E0A01236F0001D5DFF0DF82
:1005C000050E0901EC6F00019CDF030E0A01236F89
:1005D0000001CADFE5DF010E0901EC6F000191DFC8
:1005E000030E0A01236F0001BFDFDADF010E0901EC
:1005F000EC6F000186DF020E0A01236F0001B4DFF9
:10060000CFDF010E0901EC6F00017BDF020E0A0152
:10061000236F0001A9DFC4DF010E0901EC6F0001A7
:1006200070DF0E0E0A01236F00019EDFB9DF010E9D
:100630000901EC6F000165DF0A01236B000194DF03
:10064000AFDF010E0901EC6F00015BDF080E0A014C
:10065000236F000189DFA4DF010E0901EC6F0001A7
:1006600050DF0A01236B00017FDF9ADF010E0901D1
:10067000EC6F000146DF0C0E0A01236F000174DFEE
:100680008FDF010E0901EC6F00013BDF0A01236BD4
:1006900000016ADF85DF010E0901EC6F000131DF27
:1006A000060E0A01236F00015FDF7ADF010E0901E8
:1006B000EC6F000126DF0A01236B000155DF70DFBC
:1006C000010E0901EC6F00011CDF010E0A01236F0E
:1006D00000014ADF65DF020E0901EC6F000111DF46
:1006E0005FEF12F00A01236B00013EDF59DF020EBB
:1006F0000A01236F000138DF53DF020E0901EC6F9E
:100700000001FFDE61EF12F00901EC6BF2CFEDF9B1
:10071000F29EAA6AA96AA69CA69EA680A850EDBFD2
:10072000F28E4F0801E0EC2BF2CFEDF9F29EAA6AAF
:10073000010EA96EA69CA69EA680A850EDBFF28EC3
:100740004B0801E0EC2BF2CFEDF9F29EAA6A020E03
:10075000A96EA69CA69EA680A850EDBFF28E490861
:1007600001E0EC2BF2CFEDF9F29EAA6A030EA96E1E
:10077000A69CA69EA680A850EDBFF28E520801E06E
:10078000EC2BF2CFEDF9F29EAA6A040EA96EA69C9C
:10079000A69EA680A850EDBFF28E410801E0EC2B8A
:1007A000F2CFEDF9F29EAA6A050EA96EA69CA69E4E
:1007B000A680A850EDBFF28E4B0801E0EC2BF2CFE3
:1007C000EDF9F29EAA6A060EA96EA69CA69EA680C8
:1007D000A850EDBFF28E550801E0EC2B81B801D096
:1007E000EC2B81BA01D0EC2BECC901F0000163EFD6
:1007F00012F0F250006EF29EEFC9AAFFEEC9A9FFF7
:10080000F0C9A8FFA69CA69EA6840F01550EA76E50
:10081000AA0EA76EA682A6B2FED7A6940050F21228
:10082000000112000901EF6BEE6B4F0EF06F00013B
:10083000E0DF0901EF6B010EEE6F4B0EF06F000170
:10084000D8DF0901EF6B020EEE6F490EF06F000169
:10085000D0DF0901EF6B030EEE6F520EF06F000157
:10086000C8DF0901EF6B040EEE6F410EF06F00015F
:10087000C0DF0901EF6B050EEE6F4B0EF06F00014C
:10088000B8DF0901EF6B060EEE6F550EF06F000139
:10089000B0DF67EF12F00901EC5302E1899001D05B
:1008A0008980000112000901F039006E0F0E001658
:1008B00000500F0BF26FF0510F0BF16FF2C923FADA
:1008C000000152DE6DDED50E006E002EFED7F1C99E
:1008D00023FA4ADE65DED50E006E002EFED794EFB9
:1008E00004F00901ED51000A000107E0010A06E0E9
:1008F000030A09E0010A0CE010D00FD0400E0901F4
:10090000EC2700010AD0140E0901EC27000105D0E4
:10091000540E0901EC27000100D0800E0901EC25DE
:10092000EF6FF06F0001BFD712000A012039216F6D
:100930000F0E21172017100E2125226F236F0001A3
:1009400013DE2EDE100E0A012025226F236F000118
:100950000BDE26DED50E006E002EFED7120009003B
:10096000F5520CE0F6CFECF9F7CFEDF9F5CF20FA20
:10097000DCDFECC9F6FFEDC9F7FFF1D712000A0181
:100980005C515E03F3CF01F0F4CF00F05F03F3504E
:1009900000265D515E03F3500020026E000112003C
:1009A0000901F86BF8515F083FE30A015D6BF7C975
:1009B0005CFA5F6B610E5E6F0001E1DF01C0F9F967
:1009C0000901F8510124016E000E0220036E01504E
:1009D0001C0F016E000E032201C0F9F903C0FAF9E1
:1009E0000A015D6BF6C95CFA5F6B610E5E6F000118
:1009F000C6DF02C0FCF901C0FBF90901F85101246E
:100A0000016E000E0220036E01501C0FE96E000EF5
:100A10000320EA6EEFCFFBF9FAC9EAFFF9C9E9FF53
:100A2000FBC9EFFFF82BBED7000112005F0E0901D2
:100A3000F66FF65340E00A015D6BF5C95CFA5F6B37
:100A4000610E5E6F00019BDF01C0F7F90901F651ED
:100A50000124016E000E0220036E01501C0F016E76
:100A6000000E032201C0F7F903C0F8F90A015D6B1B
:100A7000F5C95CFA5F6B610E5E6F000180DF02C03A
:100A8000FAF901C0F9F9010E0901F65D0124016EC0
:100A9000000E0220036E01501C0FE96E000E0320B1
:100AA000EA6EEFCFF9F9F8C9EAFFF7C9E9FFF9C92A
:100AB000EFFFF607BED70A015D6BF5C95CFA5F6B05
:100AC000610E5E6F00015BDF1C0E09010124E96EFF
:100AD000000E0220EA6EEF6A000112000901FA6BB3
:100AE000F86BF8515F0861E30A015D6BF5C95CFAC8
:100AF0005F6B610E5E6F000142DF01C05BFA0901AE
:100B0000F8510A010124016E000E0220036E01500B
:100B10001C0FE96E000E0320EA6EEFCF5BFA5D6BEF
:100B2000F6C95CFA5F6B610E5E6F000128DF01C0E1
:100B30005CFA0901F8510A010124016E000E02203D
:100B4000036E01501C0FE96E000E0320EA6EEF5099
:100B50005B250901FA25F96FF95302E0F92D0BD055
:100B6000036AF851FB0FE96E090E0320EA6EF9C91A
:100B7000EFFFFA6B18D0F95102080BE1036AF85144
:100B8000FB0FE96E090E0320EA6EEF6A010EFA6FA1
:100B90000AD0036AF851FB0FE96E090E0320EA6ED2
:100BA000010EEF6EFA6FF82B9CD7F86BF8515F08C7
:100BB0002FE30A015D6BF7C95CFA5F6B610E5E6F34
:100BC0000001DDDE01C05BFA0901F8510A010124D0
:100BD000016E000E0220036E01501C0F016E000E0C
:100BE000032201C05BFA03C05CFA036A0901F851F1
:100BF000FB0FE96E090E0320EA6EEFCF5DFA5CCAC7
:100C0000EAFF01C0E9FF5DCAEFFF0901F82BCED76B
:100C1000000177EF06F00901F36BF26BF16B010E47
:100C2000F06FEF6B980EEE6F960EED6F800EEC6F1F
:100C3000F46BF4515F0809E31C0EF425E96EEA6ACF
:100C4000D8B0EA2AEF6AF42BF4D7F46BF4511F08FA
:100C50002BE3EC51F015006EED51F115016EEE51E4
:100C6000F215026EEF51F315036E005206E10152C8
:100C700004E1025202E1035209E04C0EF425E96E50
:100C8000EA6AD8B0EA2A010EEF6E07D04C0EF425BE
:100C9000E96EEA6AD8B0EA2AEF6AD890F037F137FD
:100CA000F237F337F42BD2D7F66B0A0EF76F000149
:100CB00077DE0901F46BF45105082AE3F56B0001B6
:100CC000B5DE0901F66B010EF76F000169DE09015F
:100CD000F56B0001ABDE0901F56B0001A7DE090130
:100CE000F56B010EF66F020EF76F0001F7D6020EDC
:100CF0000901F66FF76B000153DE0B0E0901F425B5
:100D0000F56FF66BF76F00014BDE0901F42BD3D7BB
:100D1000000197EF12F00901EC6B030EED6F00017B
:100D2000E0DD1B50010A11E0030A15E0010A19E099
:100D3000070A1DE0010A21E0030A25E0010A29E073
:100D40000F0A2DE0010A31E036D03C0EF66E040E9B
:100D5000F76E05DE32D04A0EF66E040EF76EFFDD3A
:100D60002CD0580EF66E040EF76EF9DD26D0660E06
:100D7000F66E040EF76EF3DD20D0740EF66E040EE0
:100D8000F76EEDDD1AD0820EF66E040EF76EE7DD1B
:100D900014D0900EF66E040EF76EE1DD0ED09E0EAE
:100DA000F66E040EF76EDBDD08D0AC0EF66E040EA8
:100DB000F76ED5DD02D0010E1B6E1AA206D0BA0E58
:100DC000F66E040EF76ECBDD05D0C00EF66E040E87
:100DD000F76EC5DD1AA00BD0440E0A01206F00018A
:100DE000A4DD430E0A01206F00019FDD0AD0410EF1
:100DF0000A01206F000199DD430E0A01206F0001F6
:100E000094DD12000901EC5302E1898401D0899438
:100E1000000112000E0E0901EC6F030EED6F0001D0
:100E200060DD1AA206D0010E0901EC6F000133DD6E
:100E300004D00901EC6B00012EDD1AA005D00901D8
:100E4000EC6B0001DFDF05D0010E0901EC6F000142
:100E5000D9DF12000900F6CF1EFAF7CF1FFAF5CF3F
:100E600020FA63DD1ECAF6FF1FCAF7FF0A011D2F15
:100E700001D002D00001EED700011200D8B204D098
:100E80000A0EEA6E310EE96E006A016A026A036AAE
:100E90000A01316B326B336B346B30512F112E11D1
:100EA0002D112CE0200E356FD89029372A372B379B
:100EB0002C3731373237333734373051345D08E12E
:100EC0002F51335D05E12E51325D02E12D51315D2F
:100ED0000FE32D51315F2E51D8A02E3D325F2F519F
:100EE000D8A02F3D335F3051D8A0303D345FD8803B
:100EF0000036013602360336352FD6D731CAEFFF1A
:100F000032CAECFF33CAECFF34CAECFF0001120016
:100F1000E9500901F06FEFAF0DD0F007F08BEC1F37
:100F2000ED1FEE1FEF1FEC2BD8B4ED2BD8B4EE2B3A
:100F3000D8B4EF2B3B0EF76F9A0EF66FCA0EF56F13
:100F4000F46B0A0EF26FD882090EEA6EEC0EE96EAF
:100F5000EFC92CFAEEC92BFAEDC92AFAECC929FA25
:100F6000F7C930FAF6C92FFAF5C92EFAF4C92DFAE5
:100F7000000184DF0150005213E10901F251010A1E
:100F8000D8A402D000010CD0F0510DE00F0BF25D9F
:100F900001E02DE2F0BF2BD0F0BD05D0200E21D016
:100FA000200E0901F017F0AB0CD0F09B00C0F0F957
:100FB0002D0E0A01206F0001B8DC0901F0C900F014
:100FC000F06B300EF0AB0DD0F09B00C0F0F92D0EA1
:100FD0000A01206F0001A9DC0901F0C900F0F06BE3
:100FE000300E002600C020FA00019FDC0901D892D3
:100FF000F7C92CFAF6C92BFAF5C92AFAF4C929FA65
:101000000A01306B2F6B2E6B0A0E2D6F000136DF3D
:1010100003C0F7F902C0F6F901C0F5F900C0F4F910
:101020000901F22F90D70001E4EF12F0EACFF4F9B2
:10103000E9CFF3F90901EDAF08D0F38FF3A9F32B52
:10104000EC1FED1FEC2BD8B4ED2BED39F009EF6F51
:10105000EF27E20FF06F320FF26FED510F0BF02719
:10106000F027F227E90FF16FF127F127EC390F0B89
:10107000F127F227F137F237F21FF237EC510F0B5D
:10108000F227EF37070EEE6F0A0EF107F227FDE3A6
:10109000F007F127FDE3EF07F027FDE3EE07EF2769
:1010A000FDE3090EEA6EEE0EE96E070EF315F39DF1
:1010B000ED52F31507E1F3B9EE52F3B903D0200E68
:1010C000006E21D0E926000EEA22E950F20804E180
:1010D000EA50090801E1F38DEF50006E08E1F3BD1D
:1010E00006D0F3B91DD0F3B702D0200E0BD0F3AF6A
:1010F00006D02D0E006EED50F39DF39F04D0F387C4
:10110000F399300E0026EACFEDF9E9CFECF900C0F3
:1011100020FA00010ADCEDC9EAFFECC9E9FF090188
:10112000EE50F3ADD2D7000112000901F96BFA6B52
:10113000010EFB6FDA6AD96A090EFE6FF10EFD6FC0
:10114000090EEA6EF50EE96EFEC9E2FFFDC9E1FF88
:10115000FBC9FCF9D890E550EE02F350F923F450A6
:10116000FA23FC2FF7D7F9C9DEFFFAC9F9F9FA6BB0
:10117000D8B0FA2BFD2BD8B4FE2BFB2BFB51050866
:10118000DFE100014DEF13F0B5C9EAFFB4C9E9FF93
:101190000A0129CAEFFFE92AD8B4EA2AEF6A09014D
:1011A000B42BD8B4B52B00011200E9500A01216F0D
:1011B00020AF0DD02107218B1D1F1E1F1F1F201FB9
:1011C0001D2BD8B41E2BD8B41F2BD8B4202B3B0E0C
:1011D000286F9A0E276FCA0E266F256B0A0E236F93
:1011E000D8820A0EEA6E1D0EE96E20CA2CFA1FCABA
:1011F0002BFA1ECA2AFA1DCA29FA28CA30FA27CAA7
:101200002FFA26CA2EFA25CA2DFA000137DE015020
:10121000005213E10A012351010AD8A402D00001AF
:101220000CD021510DE00F0B235D01E02BE221BF1B
:1012300029D021BD05D0200E1FD0200E0A01211774
:1012400021AB0BD0219B00C021FA2D0E296F00018C
:101250009BDF0A0121CA00F0216B300E21AB0CD0BC
:10126000219B00C021FA2D0E296F00018DDF0A019C
:1012700021CA00F0216B300E002600C029FA0001BF
:1012800083DF0A01D89228CA2CFA27CA2BFA26CA69
:101290002AFA25CA29FA306B2F6B2E6B0A0E2D6F96
:1012A0000001ECDD03C028FA02C027FA01C026FACB
:1012B00000C025FA0A01232F93D700011200EF5234
:1012C00010E0EACF1EFAE9CF1DFAEFCF20FA95EC35
:1012D00004F01ECAEAFF1DCAE9FFE92AD8B4EA2AC7
:1012E000EED71200090E0901B56FF50EB46F080EA6
:1012F000E96EF4C920FAF3C91FFAF2C91EFAF1C95E
:101300001DFA000152DFF5C909FAF6C90AFA200EE2
:101310000A010B6FF7C90CFAF8C90DFAF9C90EFAF0
:101320000F6FFAC910FAFBC911FAFCC912FA136B54
:10133000C60EF66E040EF76E060E1D6F00018ADDF6
:101340000A0EEA6E090EE96EBADFCE0EF66E040ED4
:10135000F76E040E0A011D6F00017CDD1200090109
:10136000FA6BF96BF86B010EF76FF66BF6512F08FD
:101370001EE30A015D6BF5C95CFA5F6B610E5E6F7F
:101380000001BFEC04F002C0FCF901C0FBF9090147
:10139000F6510124016E000E0220036E01501C0F55
:1013A000E96E000E0320EA6EEF6AF62BDFD7F66BCC
:1013B000F6511F0837E3F151F715006EF251F81599
:1013C000016EF351F915026EF451FA15036E0052D5
:1013D00006E1015204E1025202E103521CE00A015B
:1013E0005D6BF5C95CFA5F6B610E5E6F0001BFEC6F
:1013F00004F001C0FBF9300E0901F6250124016E4D
:10140000000E0220036E01501C0FE96E000E032037
:10141000EA6E010EEF6ED890F737F837F937FA37E2
:10142000F62BC6D7500EF66FF6515F081EE30A0181
:101430005D6BF5C95CFA5F6B610E5E6F0001BFEC1E
:1014400004F002C0FCF901C0FBF90901F6510124C6
:10145000016E000E0220036E01501C0FE96E000E9B
:101460000320EA6EEF6AF62BDFD700018BEF13F053
:101470000901EF51020A00010DE0060A10E00C0A12
:1014800017E0180A22E0300A31E0600A44E0C00A9E
:101490005BE077D0EEC9F5F916EC05F072D0EEC935
:1014A000F5F916EC05F0EEC9F5F916EC05F069D082
:1014B000EEC9F5F916EC05F0EEC9F5F916EC05F0F4
:1014C000EEC9F5F916EC05F05CD0EEC9F5F916ECAD
:1014D00005F0EEC9F5F916EC05F0EEC9F5F916ECD4
:1014E00005F0EEC9F5F916EC05F04BD0EEC9F5F9AB
:1014F00016EC05F0EEC9F5F916EC05F0EEC9F5F9B4
:1015000016EC05F0EEC9F5F916EC05F0EEC9F5F9A3
:1015100016EC05F036D0EEC9F5F916EC05F0EEC97B
:10152000F5F916EC05F0EEC9F5F916EC05F0EEC983
:10153000F5F916EC05F0EEC9F5F916EC05F0EEC973
:10154000F5F916EC05F01DD0EEC9F5F916EC05F02D
:10155000EEC9F5F916EC05F0EEC9F5F916EC05F053
:10156000EEC9F5F916EC05F0EEC9F5F916EC05F043
:10157000EEC9F5F916EC05F0EEC9F5F916EC05F033
:1015800000D0A0EF13F05F0E0901F36F0A015D6B4D
:10159000F1C95CFA5F6B610E5E6F0001BFEC04F095
:1015A00002C0F7F901C0F6F90901F3510124016EF7
:1015B000000E0220036E01501C0FE96E000E032086
:1015C000EA6EEFCFF4F90A015D6BF2C95CFA5F6B6A
:1015D000610E5E6F0001BFEC04F001C0F6F9090175
:1015E000F3510124016E000E0220036E01501C0F06
:1015F000E96E000E0320EA6EEFCFF5F9F451F55DC8
:1016000003E2010E016E0AD0F551F45D03E2FF0E14
:10161000016E04D0F307BAD7000E016E000112006C
:10162000010E0901F26FF2515F0842E30A015D6B9E
:10163000F1C95CFA5F6B610E5E6F0001BFEC04F0F4
:1016400001C0F3F9010E0901F25D0124016E000EE3
:101650000220036E01501C0F016E000E032201C018
:10166000F3F903C0F4F90A015D6BF1C95CFA5F6B31
:10167000610E5E6F0001BFEC04F002C0F6F901C01C
:10168000F5F90901F2510124016E000E0220036EEA
:1016900001501C0FE96E000E0320EA6EEFCFF5F942
:1016A000F4C9EAFFF3C9E9FFF5C9EFFFF22BBBD795
:1016B0000A015D6BF1C95CFA5F6B610E5E6F000140
:1016C000BFEC04F001C0F3F95F0E09010124016EC3
:1016D000000E0220036E01501C0FE96E000E032065
:1016E000EA6EEF6A000112000901F56BF46BF45128
:1016F0005F08D8A083D00A015D6BF1C95CFA5F6B0B
:10170000610E5E6F0001BFEC04F002C05AFA01C026
:1017100059FA0901F4510A010124016E000E022058
:10172000036E01501C0FE96E000E0320EA6EEFCF2E
:10173000F6F95D6BF2C95CFA5F6B610E5E6F0001DA
:10174000BFEC04F001C059FA0901F4510A01012467
:10175000016E000E0220036E01501C0FE96E000E98
:101760000320EA6EEFCFF7F90901F5531EE1F62DDC
:1017700006D0F75304E1010EF86FF56B15D0F62D86
:1017800005D0F72D03D0F86BF56B0ED0F65305E1BD
:10179000F75303E1F86BF56B07D0F65305E1F72D2E
:1017A00003D0010EF86FF56F1ED0F62D05D0F7535C
:1017B00003E1F86BF56B17D0F62D06D0F72D04D0AA
:1017C000010EF86FF56F0FD0F65306E1F75304E101
:1017D000010EF86FF56F07D0F65305E1F72D03D032
:1017E000F86B010EF56F036AF451F90FE96E090EFB
:1017F0000320EA6EF8C9EFFFF42B79D7F46BF451AC
:101800005F0830E30A015D6BF3C95CFA5F6B610E40
:101810005E6F0001BFEC04F001C059FA0901F451F8
:101820000A010124016E000E0220036E01501C0FFC
:10183000016E000E032201C059FA03C05AFA036A6E
:101840000901F451F90FE96E090E0320EA6EEFCF9A
:101850005BFA5ACAEAFF01C0E9FF5BCAEFFF090160
:10186000F42BCDD70001FBEF0CF00901EF6BEF512A
:101870005F081EE30A015D6BEEC95CFA5F6B610EE7
:101880005E6F0001BFEC04F002C0F2F901C0F1F993
:101890000901EF510124016E000E0220036E015078
:1018A0001C0FE96E000E0320EA6EEF6AEF2BDFD704
:1018B000300EF06FECC9F1F9EDC9F2F9000163DE09
:1018C00001C0EFF90901EF2D1AD0ECC9F1F9EDC90A
:1018D000F2F9000158DE012C10D0EDC9F5F916EC33
:1018E00005F00901F02BF0515F0802E3F05303E12A
:1018F000010E016EB1D0E9D7000143D00901EF51CB
:10190000FF081AE1ECC9F1F9EDC9F2F900013BDE7B
:101910000150FF080FE0EDC9F1F982DE0901F0077F
:10192000F0515F0802E3F05303E1010E016E94D021
:10193000E9D7000126D00901EF531FE10A015D6BD1
:10194000EEC95CFA5F6B610E5E6F0001BFEC04F0E4
:1019500001C0F1F9300E09010124016E000E0220D0
:10196000036E01501C0FE96E000E0320EA6E010E9B
:10197000EF6E000E016E70D003D0010E016E6CD0C0
:1019800000010901F0515F0802E3F05303E1010E89
:10199000016E62D0F0510F085DE2ECC9F1F9EDC9BA
:1019A000F2F90001F0DD01C0EFF90901EF2D29D0B6
:1019B0000A015D6BEEC95CFA5F6B610E5E6F000140
:1019C000BFEC04F001C0F1F90901F0510124016EEE
:1019D000000E0220036E01501C0FE96E000E032062
:1019E000EA6E010EEF6EECC9F1F9EDC9F2F9ECC93E
:1019F000F3F9000179D6EDC9F1F912DE0901F0071A
:101A000028D0EF51FF0807E1EDC9F1F9000108DE28
:101A10000901F0071ED00A015D6BEEC95CFA5F6B2D
:101A2000610E5E6F0001BFEC04F002C0F2F901C06C
:101A3000F1F90901F0510124016E000E0220036E3C
:101A400001501C0FE96E000E0320EA6E010EEF6ECE
:101A5000F06BA0D7000E016E0001A9EF13F0090191
:101A6000F16BF06BEF6B010EEE6FF56BF46BF36BDC
:101A7000F26BED6BED511F082DE30A015D6BECC9B4
:101A80005CFA5F6B610E5E6F0001BFEC04F002C098
:101A9000F7F901C0F6F9300E0901ED250124016EB8
:101AA000000E0220036E01501C0FE96E000E032091
:101AB000EA6EEF5208E0EE51F213EF51F313F051DA
:101AC000F413F151F513D890EE37EF37F037F137C3
:101AD000ED2BD0D7F2C900F0F3C901F0F4C902F040
:101AE000F5C903F00001AFEF13F00901F06BEF6BE4
:101AF000EE6BED6B0A015D6BECC95CFA5F6B610E1E
:101B00005E6F0001BFEC04F002C0F2F901C0F1F910
:101B10002F0E09010124016E000E0220036E0150F8
:101B20001C0FE96E000E0320EA6EEF5206E0650E10
:101B3000EE27CD0EEF231D0EF0230A015D6BECC9DD
:101B40005CFA5F6B610E5E6F0001BFEC04F002C0D7
:101B5000F2F901C0F1F92E0E09010124016E000E07
:101B60000220036E01501C0FE96E000E0320EA6E86
:101B7000EF5208E0800EED27B20EEE23E60EEF23C3
:101B80000E0EF0230A015D6BECC95CFA5F6B610E0F
:101B90005E6F0001BFEC04F002C0F2F901C0F1F980
:101BA0002D0E09010124016E000E0220036E01506A
:101BB0001C0FE96E000E0320EA6EEF5208E0400EA3
:101BC000ED27590EEE23730EEF23070EF0230A01C3
:101BD0005D6BECC95CFA5F6B610E5E6F0001BFEC80
:101BE00004F002C0F2F901C0F1F92C0E0901012440
:101BF000016E000E0220036E01501C0FE96E000EF4
:101C00000320EA6EEF5208E0A00EED27AC0EEE23A3
:101C1000B90EEF23030EF0230A015D6BECC95CFAE9
:101C20005F6B610E5E6F0001BFEC04F002C0F2F961
:101C300001C0F1F92B0E09010124016E000E0220F2
:101C4000036E01501C0FE96E000E0320EA6EEF5286
:101C500008E0500EED27D60EEE23DC0EEF23010E2A
:101C6000F0230A015D6BECC95CFA5F6B610E5E6F7D
:101C70000001BFEC04F002C0F2F901C0F1F92A0E34
:101C800009010124016E000E0220036E01501C0F99
:101C9000E96E000E0320EA6EEF5208E0280EED27F1
:101CA0006B0EEE23EE0EEF23000EF0230A015D6BA8
:101CB000ECC95CFA5F6B610E5E6F0001BFEC04F073
:101CC00002C0F2F901C0F1F9290E09010124016EE7
:101CD000000E0220036E01501C0FE96E000E03205F
:101CE000EA6EEF5208E0940EED27350EEE23770EE4
:101CF000EF23000EF0230A015D6BECC95CFA5F6B09
:101D0000610E5E6F0001BFEC04F002C0F2F901C089
:101D1000F1F9280E09010124016E000E0220036E64
:101D200001501C0FE96E000E0320EA6EEF5208E02E
:101D3000CA0EED279A0EEE233B0EEF23000EF02382
:101D40000A015D6BECC95CFA5F6B610E5E6F0001AE
:101D5000BFEC04F002C0F2F901C0F1F9270E09014D
:101D60000124016E000E0220036E01501C0FE96E6B
:101D7000000E0320EA6EEF5208E0650EED27CD0E4F
:101D8000EE231D0EEF23000EF0230A015D6BECC95C
:101D90005CFA5F6B610E5E6F0001BFEC04F002C085
:101DA000F2F901C0F1F9260E09010124016E000EBD
:101DB0000220036E01501C0FE96E000E0320EA6E34
:101DC000EF5208E0B20EED27E60EEE230E0EEF23E3
:101DD000000EF0230A015D6BECC95CFA5F6B610ECB
:101DE0005E6F0001BFEC04F002C0F2F901C0F1F92E
:101DF000250E09010124016E000E0220036E015020
:101E00001C0FE96E000E0320EA6EEF5208E0590E37
:101E1000ED27730EEE23070EEF23000EF0230A01C9
:101E20005D6BECC95CFA5F6B610E5E6F0001BFEC2D
:101E300004F002C0F2F901C0F1F9240E09010124F5
:101E4000016E000E0220036E01501C0FE96E000EA1
:101E50000320EA6EEF5208E0AC0EED27B90EEE2338
:101E6000030EEF23000EF0230A015D6BECC95CFA50
:101E70005F6B610E5E6F0001BFEC04F002C0F2F90F
:101E800001C0F1F9230E09010124016E000E0220A8
:101E9000036E01501C0FE96E000E0320EA6EEF5234
:101EA00008E0D60EED27DC0EEE23010EEF23000E28
:101EB000F0230A015D6BECC95CFA5F6B610E5E6F2B
:101EC0000001BFEC04F002C0F2F901C0F1F9220EEA
:101ED00009010124016E000E0220036E01501C0F47
:101EE000E96E000E0320EA6EEF5207E06B0EED275D
:101EF000EE0EEE23000EEF23F0230A015D6BECC91A
:101F00005CFA5F6B610E5E6F0001BFEC04F002C013
:101F1000F2F901C0F1F9210E09010124016E000E50
:101F20000220036E01501C0FE96E000E0320EA6EC2
:101F3000EF5207E0350EED27770EEE23000EEF236C
:101F4000F0230A015D6BECC95CFA5F6B610E5E6F9A
:101F50000001BFEC04F002C0F2F901C0F1F9200E5B
:101F600009010124016E000E0220036E01501C0FB6
:101F7000E96E000E0320EA6EEF5207E09A0EED279D
:101F80003B0EEE23000EEF23F0230A015D6BECC93C
:101F90005CFA5F6B610E5E6F0001BFEC04F002C083
:101FA000F2F901C0F1F91F0E09010124016E000EC2
:101FB0000220036E01501C0FE96E000E0320EA6E32
:101FC000EF5207E0CD0EED271D0EEE23000EEF239E
:101FD000F0230A015D6BECC95CFA5F6B610E5E6F0A
:101FE0000001BFEC04F002C0F2F901C0F1F91E0ECD
:101FF00009010124016E000E0220036E01501C0F26
:10200000E96E000E0320EA6EEF5207E0E60EED27C0
:102010000E0EEE23000EEF23F0230A015D6BECC9D8
:102020005CFA5F6B610E5E6F0001BFEC04F002C0F2
:10203000F2F901C0F1F91D0E09010124016E000E33
:102040000220036E01501C0FE96E000E0320EA6EA1
:10205000EF5207E0730EED27070EEE23000EEF237D
:10206000F0230A015D6BECC95CFA5F6B610E5E6F79
:102070000001BFEC04F002C0F2F901C0F1F91C0E3E
:1020800009010124016E000E0220036E01501C0F95
:10209000E96E000E0320EA6EEF5207E0B90EED275D
:1020A000030EEE23000EEF23F0230A015D6BECC953
:1020B0005CFA5F6B610E5E6F0001BFEC04F002C062
:1020C000F2F901C0F1F91B0E09010124016E000EA5
:1020D0000220036E01501C0FE96E000E0320EA6E11
:1020E000EF5207E0DC0EED27010EEE23000EEF238A
:1020F000F0230A015D6BECC95CFA5F6B610E5E6FE9
:102100000001BFEC04F002C0F2F901C0F1F91A0EAF
:1021100009010124016E000E0220036E01501C0F04
:10212000E96E000E0320EA6EEF5206E0EE0EED2798
:10213000000EEE23EF23F0230A015D6BECC95CFA7D
:102140005F6B610E5E6F0001BFEC04F002C0F2F93C
:1021500001C0F1F9190E09010124016E000E0220DF
:10216000036E01501C0FE96E000E0320EA6EEF5261
:1021700006E0770EED27000EEE23EF23F0230A0191
:102180005D6BECC95CFA5F6B610E5E6F0001BFECCA
:1021900004F002C0F2F901C0F1F9180E090101249E
:1021A000016E000E0220036E01501C0FE96E000E3E
:1021B0000320EA6EEF5206E03B0EED27000EEE2301
:1021C000EF23F0230A015D6BECC95CFA5F6B610ED3
:1021D0005E6F0001BFEC04F002C0F2F901C0F1F93A
:1021E000170E09010124016E000E0220036E01503A
:1021F0001C0FE96E000E0320EA6EEF5206E01D0E82
:10220000ED27000EEE23EF23F0230A015D6BECC9EE
:102210005CFA5F6B610E5E6F0001BFEC04F002C000
:10222000F2F901C0F1F9160E09010124016E000E48
:102230000220036E01501C0FE96E000E0320EA6EAF
:10224000EF5206E00E0EED27000EEE23EF23F023F3
:102250000A015D6BECC95CFA5F6B610E5E6F000199
:10226000BFEC04F002C0F2F901C0F1F9150E09014A
:102270000124016E000E0220036E01501C0FE96E56
:10228000000E0320EA6EEF5206E0070EED27000E67
:10229000EE23EF23F0230A015D6BECC95CFA5F6B60
:1022A000610E5E6F0001BFEC04F002C0F2F901C0E4
:1022B000F1F9140E09010124016E000E0220036ED3
:1022C00001501C0FE96E000E0320EA6EEF5206E08B
:1022D000030EED27000EEE23EF23F0230A015D6BC2
:1022E000ECC95CFA5F6B610E5E6F0001BFEC04F03D
:1022F00002C0F2F901C0F1F9130E09010124016EC7
:10230000000E0220036E01501C0FE96E000E032028
:10231000EA6EEF5206E0010EED27000EEE23EF23EA
:10232000F023EDC900F0EEC901F0EFC902F0F0C9E9
:1023300003F00001BDEF13F0090E0901B56FF40EB3
:10234000B46F080EE96EEFC920FAEEC91FFAEDC9A5
:102350001EFAECC91DFA0001D5EC08F0F4C908FA20
:10236000F5C909FA200E0A010A6FF6C90BFAF7C976
:102370000CFAF8C90DFA0E6FF9C90FFAFAC910FA7A
:10238000FBC911FA126B0A0EEA6E080EE96E000123
:102390005FEC09F02E0E0A01206F000195EC04F0AD
:1023A000090E0901B56FF40EB46F090EE96EF3C999
:1023B00020FAF2C91FFAF1C91EFAF0C91DFA00018C
:1023C000D5EC08F0F4C908FA0A010851200802E126
:1023D000300E086FF5C909FA0951200802E1300EE4
:1023E000096FF6C90AFA0A51200802E1300E0A6F95
:1023F000200E0B6FF7C90CFA0C51200802E1300EC9
:102400000C6FF8C90DFA0D51200802E1300E0D6F66
:10241000F9C90EFA0E51200802E1300E0E6F480E77
:102420000F6F7A0E106F116B0A0EEA6E080EE96ECE
:1024300000015FEC09F0D7EF13F0F86AD09E078E29
:10244000700ED36E9B8C9B9E1A6A1B6A09019A6B55
:10245000996B986B976B9C6B9B6B9E6B9D6BA46B46
:10246000A36BA66BA56BA86BA76BAA6BA96BAB6BD9
:10247000AC6B010EAD6FAE6FAF6BB06BB26BB16B8F
:10248000640EB36FB56BB46B0F01386B396B3A6B7D
:10249000776A786A796A700ED36E9B8C9B9EC80EA1
:1024A0000901EC6F000181EC02F096EF02F0C80E1A
:1024B0000901EC6F000181EC02F0D5EF02F072EF40
:1024C00003F084EF03F00152D8A412EF04F002EFFE
:1024D00000F0196AF2BE198EF29E050E0A01676FAE
:1024E000686B00015FEC00F019BEF28E196AF2BE53
:1024F000198EF29E0A01676B000157EC00F019BEBD
:10250000F28E0901EC6B00014BEC04F00901A66BA3
:10251000020EA56FEC6BED6B000171EC04F0D40EB4
:10252000F66E040EF76EAFEC04F00BEF06F0640EDF
:102530000901EC6F000181EC02F0C50ED56ED76A7F
:10254000070ED66EF28AC00EF212010E1B6E8BECD5
:1025500006F01A6A0AEC07F00901AB530BE0AB6B0B
:102560001B2A1B50090802E2010E1B6E00018BECB6
:1025700006F00901AC5308E0AC6B1A2A030E1A16D8
:1025800000010AEC07F0090100018BEC06F00901DB
:10259000EC6B010EED6F000171EC04F0E00EF66ED5
:1025A000040EF76E060E0A011D6F00012AEC07F0FB
:1025B000080EE96E9AC9EFF999C9EEF998C9EDF9D3
:1025C00097C9ECF988EF07F00901EC6B020EED6F8B
:1025D000000171EC04F0EC0EF66E040EF76E060EC0
:1025E0000A011D6F00012AEC07F0040EE96EA4C970
:1025F000EDF9A3C9ECF916EC08F0F60EF66E040E30
:10260000F76E070E0A011D6F00012AEC07F0020E9B
:10261000E96EA8C9EDF9A7C9ECF916EC08F00901B3
:10262000EC6BED6B000171EC04F00901975307E1CD
:10263000985305E1995303E19A53D8B4B9D01B508C
:10264000010A000111E0030A3BE0010A4EE0070A1B
:102650004CE0010A4AE0030A48E0010A46E00F0A9A
:1026600044E0010A42E0A3D0D89009019A31F06F0A
:102670009931EF6F9831EE6F9731ED6FF0C9F4F942
:10268000EFC9F3F9EEC9F2F9F16FF86BF76BF66B7E
:102690000A0EF56F000195EF08F003C0F0F902C0D3
:1026A000EFF901C0EEF900C0EDF903C0F4F902C082
:1026B000F3F901C0F2F900C0F1F972EC09F077D03A
:1026C000D89009019A31F06F9931EF6F9831EE6F20
:1026D0009731ED6FF0C9F4F9EFC9F3F9EEC9F2F9EA
:1026E000F16F000172EC09F062D0D89009019A31C3
:1026F000F06F9931EF6F9831EE6F9731ED6FF0C950
:10270000F4F9EFC9F3F9EEC9F2F9F16F010EF56FC3
:102710000001AFEF09F0030E1B5C0A0F0901EC6F1B
:10272000F66FF76B0001D0EC04F0D8900901A631E8
:10273000ED6FA531EC6FEE6BEF6F000138EF0AF033
:102740000901EC6B010EED6F020EEE6F000135EF2B
:102750000CF0020E0901EC6F00012FEF0DF003C029
:10276000BCF902C0BBF901C0BAF900C0B9F9020E48
:102770000901EC6F000175EF0DF003C0C0F902C054
:10278000BFF901C0BEF900C0BDF9BCC9EFF9BBC9B2
:10279000EEF9BAC9EDF9B9C9ECF9C0C9F3F9BFC985
:1027A000F2F9BEC9F1F9BDC9F0F9C6D500D00901E9
:0427B000D4D6030078
:020000040030CA
:0E00000000E8183C003F81000FC00FE00F40E9
:00000001FF
